:10000000A8286D306F22851DCC280108850C0319A6
:100010000328800C850C800C850C800C850C800CD2
:10002000850C800C850C800C940A850C800C850C4A
:10003000800C840A850C800C850C800C1408850CBF
:10004000800C850C800CC039850C800C850C800CD4
:10005000CD3E850C800C850C800C840A850C800CB0
:10006000850C800C850C82009834963480340F34D3
:100070004234403401348634A03400342734103400
:1000800000340334E8340034003464340034003481
:100090000A34D334C034C434CB346A2A0034013433
:1000A000043405341034113414341534D334C034CA
:1000B000CD34CF34D134D334C834CD34CF34D1342B
:1000C000043408341034203405340A341434283409
:1000D000BC345E342E3417340B340534033401340D
:1000E0004D3448347A34AF344F3466346634203477
:1000F000443469347334633468342E3420344334E4
:100100006834613472346734E53441346E346134B8
:100110006C3479347A346534F2345334653472345F
:1001200069346134EC344634723465347134753476
:1001300065346E346334F934423461347434743465
:1001400065347234F9344234723465346134EB34DA
:100150008316860183120C308600B8238610023085
:10016000E9232830CF230630CF230D30CF23403072
:10017000CF234E308F002030960005309400B523F9
:10018000D923940BBF281530D623D7238F0A960B7B
:10019000BD2884305F23CD28DB237D22563070219B
:1001A0000318D4282A21CE28110BDF28950A15120E
:1001B000B722150A7023CD2810308C06CD281118CF
:1001C0000E2A9118DC281119D4298C305F23ED28D0
:1001D0000408263A031DC62ADB23C830CF238C101F
:1001E0009F011D0A8E0073308E1905298C149F14EF
:1001F00040308E0A8E1905299F0103309E0003109E
:100200009E0D9F0D8E0BFF281E087223D723CC3026
:10021000CF2320300D196930D82337308D1C38306A
:10022000D82320300D187030D823A5225B307021E0
:1002300003181C292A21ED281119C12A911C2529EE
:100240001118EA2A8D0A8D11ED28111C282B9D0A00
:100250009D11ED28910A1119111C08009101080047
:10026000BD23DB2334296023CE237330DD234930C3
:10027000702103183E29910A111137299118432939
:10028000111CC928BC29B722111852298610030154
:10029000F123ED232030F1230614851D3029851C20
:1002A0004D29BD239B019C018B30CF231C0870235B
:1002B0003A30D121E4308F00D223D223851D312959
:1002C000940B5C298F0B5C299B0A1B08C43E031C02
:1002D0006B299B019C0A1C08F23E031C5429BC2973
:1002E0001107B623CF239C01121413140E08F03803
:1002F0008F008F0F7929010803198029901581013A
:100300002830051A3830831681008312191018100E
:1003100004308606051A9029061D18140C1193291D
:10032000061919140C158C139808031D8C17980DB9
:100330000C139908031D0C17990DF0238E0F7629C5
:100340008C1290080319A929900318081904031D99
:100350008C16050E8F008F098F0D930D031013035C
:10036000031908008F0D920D0314120303190800DE
:100370009B0B76299C0B7629BF218601BE299C0107
:100380000519851DBF29D0239C0BC0290800CF214A
:1003900035309B0ACD21CF214F309B0AD82BD72354
:1003A0005E30D8231B08702BCE230310170D9B0043
:1003B0009B0D9B07C721C721BF217D22970A1719D3
:1003C000171CE32997011708031DF921BF221430D8
:1003D00096008F0102228F0D02228F0D02220F0D37
:1003E000D923960BE9291708043C031DF9210022A3
:1003F000CD288F008F0E8F0200228F0BFC29080062
:10040000012202224B30840026309400031026186B
:100410000314800C8403940B092A0800B7221508E2
:10042000031901288F008F0B2B2A26306F22851D80
:10043000CC2801080319172A8403850C840A800C30
:1004400006308E00850C800C8E0B222A850C800CC9
:10045000940B1D2A6A2A8F0B3F2A6C22851DCC28FB
:10046000010803192E2A342A850C800C140307393D
:100470000319840A940B332A9C0B342A6A2A0F032B
:10048000303EAC228F006C22851DCC280108031958
:10049000442A8616850C800C140307390319840A34
:1004A0009519151D622A0F08960052308E00D3232D
:1004B0000000960B552A0608DF39141E20388600E6
:1004C0004E30642A632A0F088E00D223940B4A2AE6
:1004D0009C0B4A2A9701E32902309C00303094009B
:1004E00026308400283006110C1A782A3830061578
:1004F00083168100831281010800CE230D309600FF
:10050000150815071507AC229B001B0EAD221B1BFF
:100510008C1473234D309508031D4B309B1BD8233F
:100520007030DD231B08AD221B198C147323E430BB
:100530009B1D6D30D8237330D8232030D923960BE0
:100540009D2A01300C1E0430D6232A30D623170AE8
:10055000C923D7237E30D82B890003399F00831607
:10056000081483120808890A9E008C1008001430B1
:100570009700BF22D723970BBA2A1F308C058030F3
:10058000CF2B970A1719971CC62A970125301719E0
:100590001C3E97180E3E1718073E8400BF220730F6
:1005A0008F00840A000EF8230008F823D7238F0B4E
:1005B000D12A0408F93E8400CE2307308F00840A34
:1005C00000087F39E03E203E0318A530D8238F0B6A
:1005D000DF2AED2806110D190615B7232F30B82292
:1005E000263084001D08683EB6238E0094019415C1
:1005F0000D1C8D1C940A0D188D1894030D1D072BCE
:10060000051E002B851DE828051A022B0D2B051A47
:10061000072B851DE828051E092B861600008E0B6A
:100620000D2B8E00A0238E0B122BA223850C800C89
:10063000940B112B0D18800D0D1D800903108D18C2
:10064000800C840A041B041EF52AC62A9A0A1A1171
:100650006423BF21D330CF239F01A001A1018F01CB
:10066000F5309600253097001A08203E7822851D27
:10067000262B01089E001E0D8F0D0F080339023A2C
:10068000031D432B9F0A0319A00A9B30051D332924
:10069000970B372B960B392B1A0A9600960A0310E4
:1006A0009E0D9F0DA00DA10D960B4F2B8A30CF23D1
:1006B0008C239B0B2A2B1B159C0B2A2BBC299701E7
:1006C0008F003B30B822DE2B92306023CE23643083
:1006D0006E236F30DD235230D82360301A07B623E3
:1006E0008C109F019E00A101A001A501A401A301FE
:1006F00064308323031DC9230A308323C9232E308A
:100700008C18D8239B2BA2009401940A9D230318D4
:10071000852BA5231403080033308F008C11A5010D
:10072000B423A400B423A300B4238323C3230F085A
:10073000B93E031C8F2B1E08C92B9F23A523A2099A
:10074000A309A409A509A20A080022089E072308F4
:100750000318230F9F0724080318240FA007250858
:100760000318250FA10708008F0A0F088200263002
:1007700084008001840A841FB92BEF239401D023C5
:10078000940BBF2B08008C19C92B003E0319D72BE3
:100790008C150F3903191F30303ED82BC030E5239C
:1007A0008E010E17D32B8E0BD22B0800D8232030AE
:1007B00096038614E62BBF22A2308F00B423803E1E
:1007C0000318D82B7F39D823DE2B86108E00F12317
:1007D000ED230E0EF123ED23D02B0614EF2B061084
:1007E0000C080612861206138613F03986040800D8
:0E07F0000F399E00F63E031C9B2B413ED82B7A
:104200008800010001009800F40002008C00E40026
:104210002C00880064000A00880032001400D800D6
:1042200080001A00880019002800C800C00034006F
:1042300088000A006400C80060006800C800300000
:10424000D000C9001800A100800001000100140086
:1042500090001900000064000A0000002800190006
:10426000010006000900100016002E003000640056
:0A427000CC0005000E003B00950095
:00000001FF
